:020000020000FC
:100000006AC0FFB6989B39C01123B9F4B29B29C0CE
:020010000BC023
:10001600FFB6112713BF89B3807F9D9982298BBBB9
:1000260036C0962CA72CB82C662477248824CC249A
:10003600DD24EE24B29B07C0139590E093BF9EEC9F
:1000460092BF93E093BF123058F061F0143018F06D
:1000560029F49B2D08C09091690005C0992703C01B
:10006600992D01C09A2DB29992959F7089B3807F80
:10007600982B0AC09D9911C099B3907FB29B03C07B
:100086008FEF9F6002C09229812D9BBB88BB92E0B7
:10009600B29B93E095BFFFBE1895112391F4B29BD6
:1000A60010C0139590E093BF97E792BF93E093BF7C
:1000B60099B3907F9229967F812D8595859583703A
:1000C600E4CF112799B3907F9229812D8370DDCFDC
:1000D60021E02EBF2FE52DBF2FEF2ABB2BE027BB3C
:1000E60020E42BBF21E029BFC4D362E090D278D2AE
:1000F600F89463E08CD22FEF28BB2BBB71D222275A
:1001060023BB20936800C2D380F360E061F97FD2FD
:10011600989400FDDDD001FDF4D002FD4DD104FD23
:10012600DED005FDFCD009F7202F2295022B662490
:100136007724882455243324442413D093E095BF90
:10014600789455D2889400FD36D040F001FD43D016
:1001560028F002FD20D010F004D0F2CF2E3081F727
:10016600C7CF98990BC0242D6FEF26272F70222E0C
:1001760069B3607F262BB29B2BBB03C06C2C7D2CF6
:100186008E2C232D25296FEFB29968BB2627B29BAB
:1001960028BB122E089520916E002A9519F02093FF
:1001A6006E00089520917E0020936E00AAD2C8F3B7
:1001B600C1F3CED121C020916E002A9519F020936B
:1001C6006E00089520916C0020936E009AD2C8F3B9
:1001D600C1F38BD111C020916F002A9519F020939D
:1001E6006F00089520916D0020936F0085D2C8F3AB
:1001F600C1F32093790003D0989488940895989A2F
:10020600B0E0AEE822E099992D91233008F00895E8
:100216002D91662720FD626021FD6160562E269590
:10022600269520613AD020936900209179002630E6
:1002360030F09B992D919C9911C09A9918C0CD9038
:10024600DD902D91219529D0E22E2C2D219525D0BA
:10025600C22E2D2D219521D0D22E08956D912D914E
:1002660029D0C62E6D912D9125D0D62EEACF6D912F
:100276002C912F7023FD206F1DD0C62E6D91629597
:100286006F705C915295507F652B2D9122952F7042
:1002960023FD206F0FD0D62ED4CF222351F0622F0C
:1002A6002A7A60FD246062FD216064FD206466FD9B
:1002B6002061089527FD06C0222311F467FF0895E3
:1002C6006FE708952F3F11F467FD089560E80895DC
:1002D6003091750020917C0050917E0006C03091CF
:1002E600760020917D0050917F0030937700209317
:1002F6006A0050936C0050936E0020E0F3D018947F
:10030600089520917C0020936B0020917E0020931D
:100316006D0020936F006091800013D20DC0209174
:100326007D0020936B0020917F0020936D00209329
:100336006F006091810002D209F008955091740017
:10034600A6E8B0E0552309F15A952D91203CE9F035
:10035600253821F4999A5A952D91F4CF253931F4FF
:100366005A952D91203171F79B9AECCF253739F4A8
:100376005A952D91203131F02C3031F0E3CF06D053
:1003860009F308959C9A08959A9A0895237081F026
:100396002A9559F02A9531F05A9561F02D915A9582
:1003A60049F02D915A9531F02D915A9519F02D91CC
:1003B60018940895989408952091750020937700D5
:1003C60020917C0020936A0020917E0020936C008F
:1003D60020936E0060918000B4D109F00895E2EB9D
:1003E600F4E06AD029F0E8EBF4E066D009F008956D
:1003F60033273093820030938300309384005A95DC
:100406002D91253831F433955A952D9120938500F9
:10041600F6CF213A21F45A952D91223011F0989475
:1004260008955A952D912537D1F75A952D91283053
:10043600B1F75A952D91253719F1253911F40CD0BC
:10044600F8CF293011F40BD0F4CF213811F411D0A4
:10045600F0CF9CDF71F308955A950D9008955A9543
:100466002D910A943395203309F008953093820034
:1004760008955A952D91213009F00895300D08956B
:100486005A952D91213019F0243059F008955A9536
:100496002D91253909F008955A952D91243009F0AA
:1004A60001C030683093830018940895050109044B
:1004B600A10105010905A10150917400A6E8B0E06B
:1004C60036E005902D91201519F45A953A95C9F7FD
:1004D600089560918800693309F0089562E02091DB
:1004E6006800262720936800C9C0F3DFB0E0A6E8BD
:1004F60060E02C912F7009F062E02D91207F09F0C9
:1005060061E0362E2D913327662708D0622BAE3850
:10051600E0F3462E232D232B322E08955D912227BC
:10052600583591F05A3291F05C3271F028E05F5400
:1005360051F021E05A9539F022E05A9521F024E055
:100546005A9509F02227089532600895316008957A
:10055600209182002A95B0E0A6E8A20F66272D9189
:10056600203009F461602F3F09F468602D91203036
:1005760009F464602F3F09F46260462E20918300DF
:10058600622F6F77A6E8A60F6D915C9127FF08C0D2
:1005960056956795569567955695679556956795B9
:1005A6009E9906C0262F252BC9F051FD9D9A9E9A2D
:1005B6009D990BC0562F52956795652B222761FD95
:1005C600226060FD2160322E0895222765FD21609C
:1005D60061FD226051FD246062FD2860322E08957F
:1005E60032E303D03A95E9F7089544E601C04AE0BC
:1005F60003D04A95E9F7089524E6000000000000BC
:10060600000000002A95C9F7089523E0F6CF78EA9E
:100616007260DF987FB920D06FB91ED0DF9A089537
:100626007260DF987FB918D02D9115D05A95E1F7F1
:10063600DF9A0895DF987FB90FD0222715D0DF9A69
:100646000895DF987FB908D022270ED02D935A95AA
:10065600D9F7DF9A08952FB920E42EB93BE13DB9C9
:100666002EB126FFFCCF08952FB920E42EB93BE129
:100676003DB92EB126FFFCCF2FB10895F9E0EAEE81
:1006860061E08BD170E258E0CBDF60E478EEC0DF4A
:1006960020E120937000B4D009F0089560E878EE68
:1006A600B7DF2227209371002093720003C060E019
:1006B60078E3AEDF6091680070E1AADF61E078E37D
:1006C600A7DF20E220937000C6D009F408952430F5
:1006D60041F420917100239520937100283C39F74D
:1006E60009C02E3039F420917200239520937200B0
:1006F6002530E9F622230895AEE8B0E020916B009C
:1007060004C0A6E8B0E020916A0020937000A3D050
:1007160029F0243011F008940895089570E38ADFD3
:10072600522F2F9378E086DF2D935A95D9F778ECE0
:1007360064E06EDF2F91222388940895FAE0EAE0C0
:1007460009C0FAE0E2E006C0F9E0EAEF03C062E1C0
:10075600F9E0E2EF22D170E258E062DF20E1209377
:1007660070004ED009F0089578EE60E260937A004A
:100776004FDF2E912E9106D021F420EA20937000AF
:100786003FC00895A6E8B0E0209378002227209382
:10079600740020E02093700033D009F0089570E3D0
:1007A60049DF20937300522F78E044DF2D935A954A
:1007B600D9F778EC64E02CDF209174005091730037
:1007C600250F2093740020917700521730F0209166
:1007D6007400509178002517E0F222270895F9E079
:1007E600E2EEDAD0A0E6B0E070E258E019DF20E1F0
:1007F6002093700005D009F0089520E8209370003A
:100806002227209371002093720025D009F40895C1
:10081600243041F420917100239520937100283CE7
:10082600A1F709C02E3039F4209172002395209348
:100836007200253051F7263061F460917A006031FC
:1008460011F060E101C060E260937A0078EEE0DECC
:10085600E1F6222308956091700070EFD9DE78ECFE
:10086600E9DE2078E1F360E8D3DE78EFE3DE2F708F
:10087600089578E864E1CCDE78E760E2C9DE60E0FE
:10088600C7DE78E6D7DE2170E9F308953DD0D0F1D2
:1008960058EC90D054D0B1F55ADFA1F568E054DF9A
:1008A60089F56091880050DF30918A00EFE8F0E02A
:1008B6000781002309F404E020892093800024891D
:1008C6002F7020937C00268920937500208D20931D
:1008D6007E003130A1F0043091F0E8EAF0E02781A3
:1008E6002295022B20892093810024892F70209342
:1008F6007D00268920937600208D20937F006FDF70
:10090600889408950894089578ED61EC81DE78EC7A
:1009160060E27EDE78EE64E07BDE78EF8BDE207CC4
:1009260061F078ED203821F06BEC72DE689403C03C
:1009360069EC6EDEE894889408950894089528E09A
:100946002093770078EE61E063DE78EE73DE217047
:10095600E1F758EC2FD060E070EE5ADE68E0F8DE82
:1009660009F0089520918D002093770078EE61E0DC
:100976004FDE78EE5FDE2170E1F758EC1BD0F9E030
:10098600E2ED2FDF09F008955EE114D061E070EE2C
:100996003FDEF9E0EAED25CF662767FD60E807D080
:1009A60058E025912D935A95E1F75E936E93B0E04A
:1009B600A0E6089578EC60E42BDE78EC3BDE20744C
:1009C600E1F360E425DE5A95C1F7089500050100BC
:1009D600000000000009010000000000210A0000DC
:1009E600000000002109000200000100800600014D
:1009F600000012008006000200008000810600222E
:0C0A06000000800081060022010080003A
:100FC0004D535848494431207665722E332E3020D7
:100FD0002020202031362E30312E323032320D0A90
:100FE000415454696E7934342F3834202020202025
:100FF000202020202020286329206361726F0D0AA1
:00000001FF
